:020000040800F2
:1000000040080020C9000008EF000008530D000858
:1000100000000000000000000000000000000000E0
:10002000000000000000000000000000F3000008D5
:100030000000000000000000F50000084D0F00085F
:10004000F9000008F9000008F9000008F9000008AC
:10005000F9000008F9000008F9000008F90000089C
:1000600000000000F9000008F9000008F90000088D
:10007000F9000008F9000008F9000008F90000087C
:10008000F90000080000000000000000F90000086E
:1000900000000000F9000008F9000008F90000085D
:1000A00000000000F900000800000000F90000084E
:1000B0000448854600F02CFC00F05AF80048004740
:1000C00029280008400800200C4880F308880C48C4
:1000D0000168090E0B4A914205D10B480B4901609A
:1000E0000B480C4901600C4880470C480047FEE76C
:1000F000FEE7FEE7FEE7FEE7FEE70000400800201F
:10010000040000001F000000181002400100000061
:100110000000014000000000510F0008B10000087D
:1001200030B50B46014600202022012409E00D468F
:10013000D5409D4205D31D469540491B2546954017
:1001400040191546521E002DF1DC30BDD2B201E03F
:100150000270401C491EFBD270470022F6E710B522
:1001600013460A4604461946FFF7F0FF204610BD25
:1001700070B5054C054D03E0206800198047241D2B
:10018000AC42F9D170BD0000F03F0008F43F000818
:10019000F8B502464A40D40F42004B0052085B08B3
:1001A0009A4202D20246084611464A0023D0C30DA5
:1001B0004A00DDB2120EAD1A202D35DA49020126B1
:1001C000490AF6058A19002C00D0524220214F1B03
:1001D0001146B9402A411018C20D9A4221D0002C74
:1001E00017D0012D08DCDA05801AD20F8019D2074A
:1001F000DBB200F0A1F9F8BDDA05801A0123400056
:100200001B06C01880185A428018CA0F10434900B4
:1002100007E04908C2071143DA05801A801940082F
:10022000801800F081F9F8BD61000122511A001B0D
:10023000F7E70122D2075140AAE70122D207504036
:10024000A6E7024670B54A40D30FDB0740002DD029
:100250004A002AD0010E140E000212020919400AA7
:10026000520A8418E50104465443000A120A2E0477
:100270005043A4194219200CC543AA18120C012599
:10028000AD03521C521912047F39240400D0521CB1
:10029000104301D44000491EC2B20C06C009201808
:1002A000401C4008802A02D003E0002070BD4008B6
:1002B0004000002900DA0020184370BD70B50246E6
:1002C0004A40D50F40004A00ED0740085208002878
:1002D00014D0002A12D0C40DD30D41020120C00554
:1002E0005202490A520AE41A091812187D3491423E
:1002F00001D3641C00E04900002C01DA002070BD2D
:100300000023914201D3891A034340084900002881
:10031000F7D100290AD0914202D10121C90705E095
:10032000914201D2012101E00121C943E005C01839
:10033000401900F0F9F870BD420005D04200120EDD
:1003400052428A4201DB00207047C90508187047F5
:10035000F0B51FB488B00B9909980024484009995A
:10036000C00F490049080991C0070B990090490046
:1003700049080B9109990898A64608431CD00B9987
:100380000A98084318D0099801244000420D4800FB
:10039000410D099824050003000B204309900B9898
:1003A0000003000B20430B9050181C4940180022FA
:1003B00001901446104605E0002001460DB0F0BD46
:1003C000032801DA034600E003239C46C11A0AAE63
:1003D0000AE05F0008ADED5B4F00F75B7D4300274F
:1003E000AA187C41491C5B1E6145F2DD410004AB4B
:1003F0005A522104120C0A43240C401C0828DFDB4B
:10040000019802900099704601910090059B049A12
:100410000799069800F0D6F8D0E700000DFCFFFF22
:10042000C217C10F504010B54018CA0796230021CB
:1004300000F082F810BD10B500229623114600F09E
:100440007BF810BDC20F410040020123400ADB05CA
:10045000D207090EC0187F2901DA002070479629BB
:1004600003DC9623591AC84001E096398840002AD7
:10047000F4D040427047C20FD207400040080BD072
:10048000C10D0723DB01C91840020905400A1143C9
:10049000C208400711437047002001467047000022
:1004A00010B5002904DB0124E40740428C412146B9
:1004B000002B04DB1C460123DB075242A341994277
:1004C00000D1904210BD0000CB0FDB07490010B5F2
:1004D000490802460A4307D00A0D07240903E4012C
:1004E000090B121B002A01DC002010BDC900440FBB
:1004F0000C43C100E018D205801800F015F810BDBB
:100500000122D207002800DB101A002900DB511A53
:10051000814270470122D207002800DB101A00290F
:1005200000DB511A88427047002904DA401C490058
:1005300001D140084000704770B40024050C05D17B
:100540001024000402D1002921D01124050E01D16C
:1005500000020834050F01D10001241D850F01D1CF
:100560008000A41C002801DB4000641C002908D086
:1005700020252E1B0D46F540A14000D00121294326
:10058000084301061B1B000ADB1D02D5002070BCBE
:100590007047DB05181880180029F8DA401C49005C
:1005A000F5D170BC40084000704710B5002B08DA48
:1005B0000024401C614192185B411A4301D140085C
:1005C000400010BDF0B51FB482B005460C0003D04A
:1005D000084600F0F5FD02E000F0F2FD2030024692
:1005E00000902146284600F0A5F9049B059A044690
:1005F0000F4618431143084314D0184610431BD02C
:10060000009840210A1A1846059900F0A3F90546FA
:100610000E46009A0599049800F08CF9084305D01D
:10062000012004E02046394607B0F0BD0020C11784
:1006300005430E432C43374300990E986305401A37
:100640007905E40A00220C43FD0A0A3002D5002095
:100650000146E9E70105101969410C9C0D9D00193F
:100660006941FFF7A2FFDFE7F0B5074608465840AB
:1006700087B0C00F049048000E4659004008490852
:10068000BC1A884105D2384631461E4617460B46ED
:1006900002465800400810434CD0300D03904005EE
:1006A0005900400D490D0590401A0290402872DA19
:1006B00018030121000B09050843019004980092DA
:1006C000002805D0019952420020884100920190F3
:1006D000029840210A1A0199009800F02BF905466A
:1006E0000C466B4607CB00F046F9C0197141039ADE
:1006F0000E0D0023D71756401A467A40164344D0B1
:10070000049A002A2DD0029A012A039A15DC1205B8
:10071000C01A914101263605001C7141D20F059E79
:10072000D2070093019202962A462346FFF74AFF1A
:1007300007B0F0BD38463146FAE71605224A0F46A3
:10074000B218C01AB74101210905001C4F41001819
:100750007F41114618187941E20F10436D19644129
:1007600013E0E2076D0815436408C2071443039AB7
:1007700001261205C01A91413605001C7141CE07B1
:10078000400830434908C01851412A462346FFF724
:100790000CFFCDE7FFE7049801224000C117121AB1
:1007A00000238B4104983146C417381AA141EEE763
:1007B00030B40124E407634030BC55E730B4012471
:1007C000E407614030BC4FE70000E0FFF0B50C46A5
:1007D0005C4085B0E40FE40703944C0000266408F5
:1007E00059009446490802460296224321D06246A7
:1007F0000A431ED06200570D4A000E032303550D15
:10080000012402462C492405781B1B0B360B40188B
:1008100023432643614600901C46501AB44103D33B
:100820000098401C009002E0921800985B4100285C
:1008300003DA0020014605B0F0BD002001210905C2
:100840000746864611E064461D46141BB54106D393
:100850006546521BB341744607430C43A646CD0779
:1008600040084908284392185B4105460D43EAD1E8
:100870001046184313D06046194650407140084353
:1008800006D06046101AB34106D20122002306E0CA
:1008900000220123DB0702E00122D243531000981B
:1008A00074460105381C6141029C039D0019694191
:1008B000FFF77BFEBFE70000FD03000070B54B00B3
:1008C0005B0803430BD04B005C0D002633466542AA
:1008D000B341D417AD1AA34102DB0020014670BD1D
:1008E00012053018514170BD0EB5C217C10F5040EE
:1008F000CA0740180021054B0293019200910A4655
:100900000B46FFF75FFE03B000BD0000330400009C
:10091000064C0125064E05E0E36807CC2B430C3C52
:1009200098471034B442F7D3FFF7C6FBD03F000816
:10093000F03F000810B5202A04DB0146203A914020
:10094000002010BD914020239C1A0346E340194328
:10095000904010BD10B5202A04DB0846203AD04054
:10096000002110BD0B46D340D0402024A21A914054
:100970000843194610BD10B5202A06DBCB170846E0
:10098000203A1041C1170B4306E00B461341D040FB
:100990002024A21A91400843194610BDFEB5002339
:1009A0001A461B1A8A4103DB0020014603B0F0BD42
:1009B0004A000D0301212D0B0905520D0D43D107EE
:1009C00002D100186D41521E5110FF31FF3101312B
:1009D000002704463E463846009701910246012111
:1009E00000200905FFF7B6FFC3197141F818324618
:1009F00084468E464A4161462846611A904104D396
:100A00006046241A954176461F46241900986D4188
:100A1000401C00903428E1DDF91930467041091B73
:100A2000A84103D20022D243134601E0002213461C
:100A300001980105381C7141FFF7B7FDB6E770B5A5
:100A40008C180578401C6B075B0F01D10378401CA4
:100A50002A1106D10278401C03E006780E70401C73
:100A6000491C5B1EF9D12B0705D40023521E0DD45F
:100A70000B70491CFAE70378401CCB1A921C03E068
:100A80001D780D70491C5B1C521EF9D5A142D8D3AC
:100A9000002070BD836A0B43836242617047002966
:100AA000816801D0012200E0022211438160704779
:100AB0000029C16802D00122114301E04908490020
:100AC000C1607047C26802239A43C260C2680A4389
:100AD000C2607047826800210123DB071A438260ED
:100AE0000F231B038268491CD20FD207994201D001
:100AF000002AF7D18168002901DB006C70470020D3
:100B00007047000030B5C268084B8C681A400B680B
:100B10000D792343CC686D032C4323430C69496949
:100B200023430B431343C36030BD000003D2FFFFD8
:100B300081680422114381607047002101600171C6
:100B40008160C16001614161704700000122054977
:100B500092050028886801D0104300E09043886027
:100B600070470000002701400029016802D00122DF
:100B7000114301E0014A114001607047FEFF00008F
:100B800030B503680C4A0C6A13408A684D692243E9
:100B90000C692C4322438C692243CC6922434C6A62
:100BA00022438C6A22431A430260CA6842600A6880
:100BB00082604968C16030BD0F80FFFFF0B50B2730
:100BC00006463F04384600F067F804280FD1084C69
:100BD000206902252843206166612069402108437D
:100BE0002061384600F058F82169A9432161F0BD21
:100BF0000020024008490420CA68D20701D0012021
:100C00007047CA68D20601D502207047C9684907F3
:100C1000FBD5032070470000002002400248016914
:100C2000802211430161704700200240F8B506465A
:100C300000200B273F0400900D46384600F02CF8AA
:100C4000042815D10B4C206901210843206135800F
:100C5000384600F021F8042806D1B61C290C00966D
:100C60003180384600F018F82169490849002161AF
:100C7000F8BD00000020024004480169090603D5C0
:100C80000349416003494160704700000020024071
:100C900023016745AB89EFCD00B50346FFF7AAFFF7
:100CA00002E0FFF7A7FF5B1E012803D0002B00D155
:100CB000052000BD002BF4D1FAE7F0B50022032592
:100CC00001230C6893401C409C422AD10C79012CD2
:100CD00001D0022C12D1876854002E46A640B7439B
:100CE00087604E79A64084682643866084889C434A
:100CF000848084888B7993401C43848006685300E9
:100D00002C469C40A64306600E7907689E403E43F1
:100D10000660C668A643C660CC799C40C3681C4385
:100D2000C460521C102ACBD3F0BD4B07DB0E9A4097
:100D3000C90810B589000818016A0F249C40A14316
:100D40000162016A1143016210BD01857047816132
:100D50007047052000F0D0FF0029016802D0012271
:100D6000114301E0490849000160704701229203E4
:100D70000029416801D0114300E091434160704770
:100D80000246926900200A4200D00120704700000C
:100D900010B502685208520002600268134B8C685A
:100DA0001A4024024B681443234303600F230A684C
:100DB0001B069A430261026801231A430260002263
:100DC0008260C2600B698A691A438260826801236B
:100DD000DB031A438260CA680368134303604268F6
:100DE000034B49691A401143416010BDFFE0CF0039
:100DF000FF7FFF07406AC0B2704781627047000002
:100E000070B5049D44688905890D1204034E114391
:100E10001943344029432143416070BD009800FCD0
:100E200070B5FF2500210446AD05C943FFF784FADC
:100E300006460F4960100C1A21463046FFF701FAAA
:100E40002146FFF7FEF92946FFF7F7F92146FFF79C
:100E5000F8F9044601463046FFF7F3F92146FFF75B
:100E6000F0F92946FFF7E9F92146FFF7EAF970BDE5
:100E7000DF59375F044A0029516901D0014300E07E
:100E8000814351617047000000100240044A00296C
:100E9000D16901D0014300E08143D1617047000076
:100EA00000100240044A0029916901D0014300E08A
:100EB00081439161704700000010024004490A6BB1
:100EC00010239A430A630A6B02430A6370470000C7
:100ED00000100240044A0029116801D0014300E0DB
:100EE0008143116070470000000001400CB50020F4
:100EF0000090019013491120086013484168416037
:100F00004168416041687B22D2039143416041685E
:100F10000522D204114341600168012212061143E7
:100F2000016001688901FCD5416889088900416038
:100F3000416802221143416041680907890F022973
:100F4000FAD10CBD002002400010024070470000A2
:100F500010B5144801680122114301604168124A2A
:100F6000114041600168114A11400160016801228D
:100F700092049143016041683F2212049143416011
:100F8000C16A09090901C162016BFF225432914310
:100F90000163416B49084900416300218160FFF70B
:100FA000A5FF10BD001002400CB8FF08FFFFF6FEC1
:100FB0000029018802D00122114301E049084900BB
:100FC0000180704740300029818803D00122D2037C
:100FD000114301E04904490C8180704770B5028CCF
:100FE000520852000284048C8288038B7025AB4324
:100FF0009B080D889B001D4302239C438E894B88D0
:101000002643104C3343A04208D00F4CA04205D0D9
:101010000E4CA04202D00E4CA0420DD10824A34396
:10102000CC891C4304239C438B882343094C2240D6
:101030000C8A14434A8A224382800583896841636B
:10104000038470BD002C0140004001400044014079
:1010500000480140FFFC000070B5028C10239A4349
:101060000284048C8288038B1A4D2B400D782D0648
:101070002D0C1D4320239C438B891B051E0C4B8884
:1010800026431B051B0C144C3343A04202D0134EC5
:10109000B04219D1124E32400E8AB604360C324399
:1010A000A04211D18024A343CC892405240C1C43E5
:1010B00040239C438B881B051B0C2343094C224077
:1010C0004C8AA404240C22438280058389688163AE
:1010D000038470BDFF8C0000002C014000400140E3
:1010E000FFFB0000FFF7000030B5028C124B1A40E6
:1010F0000284058C8288838B104C23400C78240654
:10110000240C1C430E4B1D400B7B1B071B0C2B435D
:101110008D782D072D0C1D430A4B984205D10A4BA3
:1011200013400A8A9205120C1A43828084838968CC
:101130000164058430BD0000FFEF0000FF8C00005B
:10114000FFDF0000002C0140FFBF000010B5028847
:10115000144B984206D00124A407A04202D0124C9E
:10116000A04203D17024A2434C8822430F4CA042DA
:1011700003D00F4C22400C89224302804A68C2628D
:101180000A880285984208D00A4A904205D00A4A45
:10119000904202D0094A904201D1897A0186012108
:1011A000818210BD002C014000040040001000406E
:1011B000FFFC0000004001400044014000480140A5
:1011C0002021020C01D010211046020A01D0104645
:1011D0000839020901D01046091F820801D01046C3
:1011E000891E420801D0881E7047081A7047000007
:1011F0004900CA020243100000D004204A0D01D069
:1012000001221043044A490D914201D102210843B1
:10121000012800D105207047FF070000F8B50446FB
:101220004F1EC8000838211815461E460868496830
:101230003A4606239A4310D02A463346FFF788F8E9
:101240003A46D200083AA3181A687F1E5B68FFF777
:101250000BFA06223B469343EED1022F23D0042FF4
:1012600011D0062F2FD12A463346FFF771F8E36AD3
:10127000A26AFFF7F9F92A463346FFF769F8636A6D
:10128000226AFFF7F1F92A463346FFF761F8E3696E
:10129000A269FFF7E9F92A463346FFF759F863696F
:1012A0002269FFF7E1F92A463346FFF751F8E36870
:1012B000A268FFF7D9F92A463346FFF749F8636871
:1012C0002268FFF7D1F9F8BD002210B51346104689
:1012D0000149FFF77BFA10BD0000F03F10B5FFF7A2
:1012E000C3F910BD002210B5134610461146FFF792
:1012F0006DFA10BD10B50721024A00200907FFF75B
:10130000DDFA10BD01030000034A10B500201107EB
:10131000FFF7D4FA10BD000001FDFFFF02E008C88E
:10132000121F08C1002AFAD170477047002001E05F
:1013300001C1121F002AFBD170470000014908605B
:1013400070470000E401002001480021016070475F
:1013500014010020F8B5154E45200006374600253B
:10136000183FB06002F08AFB0024A00039588019B1
:101370000F4A01F01EFA641C032CF6DB00F0D2FECB
:10138000FF20F5306D1C8542ECDB45210906B06875
:10139000FEF74FFF074D0024B060A00080192946DA
:1013A00001F0F4F9641C032CF7DBF8BD8C0300207A
:1013B0001F856B3F0000FA4370B592B020250320D3
:1013C0006946069508770024CC77092006A9C0064F
:1013D000FFF773FC01214802FFF764FD0121084675
:1013E000FFF748FD2A4806902A48079002200990F6
:1013F00080200B9040000C90089480000E950D907A
:101400000A94C000244D0F9006A910942846FFF7B7
:10141000B7FB1F4E0221403E3046FFF753FB012130
:101420003046FFF745FB6846FFF787FB012069461A
:101430000094087104200590029404943046FFF74C
:1014400061FB0121072249043046FFF723FB0722F5
:1014500020213046FFF71EFB0120FFF777FB3046C7
:10146000FFF738FB01213046FFF719FB3046FFF745
:101470005FFB01212846FFF777FB08480088FEF74D
:10148000DAFF0749FEF7DDFE0249486012B070BD81
:10149000402401408401002008000240BAF7FF1FE9
:1014A00062DB963F10B50B49002803D0012808D015
:1014B000002010BD0888FEF7BEFF0749FEF7C1FEF9
:1014C00010BD4888FEF7B7FF014602484068FEF7A6
:1014D000F5FE10BD840100203FC8B23A70B5FF256B
:1014E0000024F53502F042FA284600F068FB641C3F
:1014F0000A2CF7DB00F006F801480168416070BD76
:101500000000002010B502F031FA0C480068FEF728
:10151000B2FF0B4A0B4BFEF71BFF0B4A0B4B01F0C4
:101520007DFCFEF7D1FF7F21C905FEF786FE084945
:10153000FEF787FE0749086010BD0000DC010020AF
:101540009A82640281B2E43E24D1CB28965BC83FE4
:10155000002A2D4700000020F8B5840013481349E5
:101560001830075909683846FEF76BFE0F4D0646DE
:1015700010352846103001593846FEF75AFE2946E4
:1015800008390968FEF75DFE09490968FEF759FE4A
:101590003146FEF752FE2851284610300751601997
:1015A000044901F0F3F82859F8BD00001C0100209F
:1015B000500100200000B44370B5002506462C46BB
:1015C000A00030580146FEF73CFE2946FEF7E0FD3C
:1015D000641CE4B20546032CF2D3FFF721FC01465C
:1015E0007F20C005FEF76AFE70BD0000F8B5164FFB
:1015F0000C227968134E5143144A8A1839688C00BA
:101600001159002802D0124E491C00E0491E115108
:10161000BD6831462859FEF714FE28513C68002C5D
:1016200004D131466868FEF70CFE686078680C21CA
:10163000484306494018A1004058002800DA4042BB
:10164000F8BD00002EBA683F44010020C00300200E
:10165000CDCC8C3F30B5002207239C1A6418203C67
:10166000855CE47FA54201D0002030BD521C072AD2
:10167000F3DB012030BD0000F0B585B0072002F09B
:1016800004FC0007400F0026072801D0022000E0DC
:10169000304601273F4D002816D02868002823D067
:1016A00000F040FD044601F0DDFA0F213A4802F057
:1016B000D6FB00F017FA002806D0EE602E616868AD
:1016C000AC61AE60EC61286200F02CFD0446A869B4
:1016D0003249201A884233D92968002930D0AC61B8
:1016E0002869002826D027E00F212B4802F0B7FBFD
:1016F00029480168A429E7D1264C017E14342170C1
:10170000017F6170018CA170818CE1704168009152
:1017100081680191C1680291016903914069049057
:10172000684602F0D4FB6868215C252002F0BEFB0D
:101730002F60C9E7286A686001F094FA2F611CE005
:101740002969002919D1E9680091052915D229686C
:10175000002912D07D21C90088420ED9FF301049DE
:10176000F530FEF7DDFC01460098401C814204D3B1
:1017700001F078FAE868401CE860E8690949201A35
:10178000884205D90848AF60066046608660C6603A
:1017900005B0F0BD94000020380300207837000029
:1017A000E40C000040420F0010030020F0B5B64FDB
:1017B0007F26B878F60585B0002801D13F26360689
:1017C0000024B248A50040593146FEF73AFDB04921
:1017D000641C4851032CF4DBAE4C01252068002624
:1017E00000283AD000F01CFC002836D0AA49012875
:1017F0000FD0042821D0032822D0072800DBA560C1
:10180000052820D0062821D0072822D0082874D007
:1018100023E0A068002809D00D60A66000F040FB1E
:1018200000F0FCFA00F07EFC9C4915E000F09AFC08
:10183000FFF790FDFFF752FEF0E73D710D600CE001
:101840000D603E7109E001F0F1F958E001F0E0F9B6
:1018500055E000F011FF52E0086001F0CFFA8A482D
:101860000079002803D08E48006800282AD08848D4
:101870008C490068FEF7E5FC8B49FEF7E2FC8B4FD4
:101880003968FEF7D6FC82490C39086080488549E2
:101890004068FEF7D6FC8449FEF7D3FC7968FEF772
:1018A000C8FC7B490C39486079487E498068FEF75E
:1018B000C8FC7D49FEF7C5FCB968FEF7BAFC74495F
:1018C0000C398860002001F0F1F9012001F0EEF9F7
:1018D000022001F0EBF96D487549C0680027884285
:1018E00005DBFEF7A6FC7349FEF7ABFC0746724822
:1018F0000068002808D104E0FFE700F05BF96F49B9
:10190000AAE76F48874215DA6068002807D000F020
:1019100009FC6168401A6B49884200D9666000275B
:10192000F8B2002101F0F2FF7F1C032FF8DDE66022
:10193000256062E0574C0020206000F0F3FB6060FF
:1019400061480068002801D06048C768604C38468C
:1019500026683146FEF76DFC049065682946FEF75F
:1019600068FCA4682146FEF713FC03903146384614
:10197000FEF70EFC06462946FEF75BFC2146FEF705
:1019800058FC019029460498FEF702FC2146FEF718
:1019900050FC029030462946FEF7FAFB2146FEF73E
:1019A000F7FB00900020401C0328FCDD0020394F8D
:1019B00004466E46F860A500705901F003F901462F
:1019C000E0B201F0A3FF70590121C907884202D992
:1019D0000020705104E07F21C905884200DD71516B
:1019E0007159F868FEF7D4FB641CF860032CE2DD43
:1019F0000121C943FEF7A0FCF860234800790028C4
:101A000040D02748006800283CD102F041F9204826
:101A100024498068FEF715FC2349FEF712FC0546B1
:101A20002C4C29466068FEF70CFC009001212068D0
:101A3000C90748402946FEF704FC01902946A068E2
:101A4000FEF7FFFB124F0025184E0C3F0290224874
:101A5000AC0001592148224A201800F0AAFE28466D
:101A6000FFF77AFD69460959FEF792FB3159FEF7F7
:101A7000E0FB6D1C3851012DE9DDB1680298FEF7DD
:101A8000D8FBB86005B0F0BD440200201003002070
:101A9000F40100202C0000205000002070000020E5
:101AA000F00000200000B44335FA8E3C8003002093
:101AB000CDCCCC3DE4388E3F9C000020540000206B
:101AC0006F12833A40420F00F8000020B00300205C
:101AD000F0030020E4000020A403002034010020D3
:101AE000A7373D3FF8B52D4C2068A52853D10021DC
:101AF00008468200A258401C51180E28F9DBC8B2D3
:101B0000A16B884247D12548103001F0BFF8244D21
:101B100028602248183001F0B9F868601F48283062
:101B200001F0B4F8A860208C616A8007800D40182D
:101B3000FEF776FC1B49FEF784FBE860207B1A4D1C
:101B40000006C00FA871A068C106C90FE97181061F
:101B5000C90F29720107C90F29706168FA2918D0C5
:101B6000002169708107C90FC007A970C00FE87014
:101B700000200E4B0E4C074601261F54225C295CA8
:101B80008A4200D01E542154401C0A28F5DB012053
:101B9000F8BD0121E5E70020F8BD00003803002072
:101BA00010030020F7FF7F3A440200202C0300209E
:101BB0002003002010B50020FFF718FD10BD08B568
:101BC000810040180090411E009101D30846FAE7B9
:101BD00008BD0000F8B5244C606AFEF721FCE16AFC
:101BE0000091FEF72EFB0546E069FEF719FC294639
:101BF000FEF7CEFA0546206B00990646FEF721FB5C
:101C00002946FEF71EFB0746A069FEF709FC314690
:101C1000FEF717FB0646A06AFEF702FC0099FEF7E6
:101C200010FB0546206AFEF7FBFB2946FEF7B0FADB
:101C30000099FEF706FB05466069FEF7F1FB2946B1
:101C4000FEF7A6FA0099FEF7FCFA05462069FEF7B2
:101C5000E7FB2946FEF79CFA3146FEF799FA39462A
:101C6000FEF796FA6063F8BDA80100203EB5082192
:101C7000762000F03DFC1E4D1E4C810616D5032338
:101C80006A461946762000F02FFC0098019900045E
:101C9000090208430299084300020012FEF7C0FB44
:101CA0002946FEF7CEFA0122206017E0C00619D5BA
:101CB00003236A460021762000F016FC0098019963
:101CC0000004090208430299084300020012FEF7CB
:101CD000A7FB2946FEF7B5FA0222606008217620AC
:101CE00000F00AFC206820636068E0623EBD0000EE
:101CF00025499234A801002006460024E0B20021C4
:101D000001F004FE641C032CF8DD0B4DAF00002431
:101D10000CE0FF2000F028FD2846FFF750FFFF20D1
:101D200000F010FD2846FFF74AFF641CB442F0DBC8
:101D30003846FFF744FFEAE7400D030010B50349BA
:101D4000FEF726FA00F004F810BD0000DB0FC93FD3
:101D500070B50446134E144D03E03146FEF718FAF1
:101D60000446AC42F9D8114DAC4204DD3146FEF7D1
:101D700060FA0446F8E70120C0070D490D4D844282
:101D8000204605D9FEF75DFA2946FEF701FA04E080
:101D9000FEF757FA2946FEF750FA2146FEF751FAA8
:101DA00070BD0000DB0FC940DB0F49C0DB0F4940AD
:101DB0007B81CF3E83F9A23FFEB500273D4600243C
:101DC000681CFEF72DFB01900E49A8000E58601C00
:101DD000FEF726FB0090A10071580198FEF731FA3A
:101DE0000099FEF72EFA0849FEF72BFA3946FEF75E
:101DF000CFF9641C0746032CE9DB6D1C032DDEDBE9
:101E0000FEBD0000780100208D976E3F10B5FFF7F2
:101E1000D3FF0149086010BD74000020F8B5002010
:101E2000012400F08FF81A4DA84230D1FF2000F0B5
:101E300089F8A8422BD12046022500F08BF81549DD
:101E400048600968FEF75CFB11D100260024B7004A
:101E500028466D1C00F07EF80F49A200C959641C89
:101E60008850032CF4DB761C032EEFDB00E00B25FF
:101E700028466D1C00F06EF8084C206028466D1C4A
:101E800000F068F86060284600F064F8A060F8BDD3
:101E90000100AA1274000020780100208C030020A9
:101EA000F8B500F05BF800F03BF800200124184979
:101EB00001F0BAFF174920460225096800F052F8E0
:101EC00000260024B7001448A100C05941582846F4
:101ED0006D1C00F047F8641C032CF4DB761C032E09
:101EE000EFDB0E4C28466D1C216800F03BF86E1CA1
:101EF0002846616800F036F83046A16800F032F8F4
:101F00000349FF2001F090FF00F018F8F8BD000031
:101F10000100AA1274000020780100208C03002028
:101F200010B50548FEF74AFE042803D0FEF776FEFA
:101F3000012010BD002010BD007C000810B5FEF788
:101F40006DFE10BD02498000401800687047000017
:101F5000007C000800B5FFF7F5FF00BD10B5FEF7E7
:101F60008BFE10BD10B501F05FFF10BD30B52A4CDF
:101F7000217881424ED007216218203AD27F6254E4
:101F8000491E0129F8DA207024492348FFF762FB33
:101F90007F25002802D06570032030BD1F491E48F0
:101FA000C91DFFF757FB002802D06570042030BD23
:101FB0001A4919480E31FFF74DFB002802D0657011
:101FC000012030BD154914481531FFF743FB0028A7
:101FD00002D06570052030BD10490F481C31FFF755
:101FE00039FB002802D06570062030BD0B490A4835
:101FF0002331FFF72FFB002802D06570072030BD8A
:10200000064905482A31FFF725FB002802D06570F4
:10201000082030BD002030BD8C000020F23E0008BA
:1020200070B53748374C0068002864D0364B3748C5
:102030001A685100490881420BDA9D686D006D08ED
:10204000854206DA5D686D006D08854201DA002080
:102050002FE02F4DAA4202D89E68AE4206D95E6894
:1020600076007608864201DA012022E0294EB2424B
:1020700002DC9A68B24206DD5A6852005208824277
:1020800001DA022015E05A68AA4208D9814206DA2C
:102090009D686D006D08854201DA032009E0B242B7
:1020A00008DD814206DA996849004908814201DA6F
:1020B0000420206000F036F806CC083C914200D0A5
:1020C000E060E268801A144A90420FD9002904D1D6
:1020D000124A904201D90C2005E0114A904204D9DD
:1020E0007F2903D0FF20A06000E0A1606160A068AC
:1020F000FFF73CFF70BD7F20A0606060002070BDD6
:102100002C0000207C00002010030020CDCC4C3E91
:10211000333333BF3333333FA086010040420F00D7
:1021200020A1070010B501F067FE10BD1CB52320EB
:1021300001214004FEF79EFE01206946087100203F
:102140008871C8710320487104200924E4060090B6
:102150002046FEF7B2FD0821009169462046FEF7B1
:10216000ACFD1CBDF0B591B0FFF7DCFF0F9005464C
:102170000B900A9000208100574B0CAA5B58401C22
:1021800053500328F7DB8DE00A980A95281A099026
:1021900001D10120099006236A464321682000F0FE
:1021A000A3F9009801990002401800B2FEF738F92F
:1021B0000790029803990002401800B2FEF730F928
:1021C0000690049805990002401800B2FEF728F91D
:1021D000424E0890307800F061FA20464049FDF701
:1021E0009FFF4048814201D9012100E00021306871
:1021F000C207D20F914201D0401C306037480178AD
:102200000907090F00260160B4000CAF06A8395970
:102210000059FEF77FF904D238593349FDF7B8FF6A
:10222000385106A839590059FEF76AF904D23859CD
:102230002D49FDF7FEFF3851E0192C4900F0A6FAB0
:1022400038592B4940004008FDF7A2FF014606AF70
:10225000385940004008FEF75DF906D2FFF762FFEB
:102260000B901E48012101600BE00998FEF7E3F88E
:10227000204900F0B4FA024617483959201800F0F6
:1022800098FA761C032EBFDB7D24E400FFF74AFF9B
:10229000401BA04203D20A20FFF791FCF6E7FFF7AC
:1022A00041FF05460B982C1A1348844205D20F981B
:1022B0001249281A884200D266E70B98291A0E485C
:1022C000814207D20020044A01468300401CD150BD
:1022D0000328FADB11B0F0BD98030020CC000020E9
:1022E00024F40000127A0000CDCCCC3D000048441C
:1022F0000000C8420024F44880841E00C0E1E400CD
:1023000010B58AB002206946087101208871C87131
:10231000032040020924E40600902046FEF7CDFC8D
:10232000042209212046FEF700FD04220A2120464E
:10233000FEF7FBFC01214805FEF7A8FD0121084638
:10234000FEF7B0FD01218805FEF7C4FD0121C80597
:10235000FEF7C0FD1020FEF7B1FD0B4802900020F3
:102360000F2104910390AB21084C05900790069132
:10237000089002A92046FEF70BFD01212046FEF73A
:10238000EBFC0AB010BD00001808700000540040BB
:10239000F8B517461E460446012200F03BF8092016
:1023A000800200906004010C0123F2B25B06124827
:1023B000FEF726FD114D0020287018E0002408E0EB
:1023C000641C600B05D00E490868401C08600020A2
:1023D000F8BD04210848FEF7D3FC0028F0D00648D9
:1023E000FEF708FD29788A00B850491C2970287822
:1023F000B042E3DB0120F8BD00540040A4010020FE
:102400008C01002008B501236A46FFF7C1FF009840
:1024100008BD0000F7B582B0174600241C4D1D4EC4
:1024200002E0641C600B24D10121C9033046FEF791
:10243000A7FC0128F5D00120400300900298FAB2D1
:102440004004010C00233046FEF7DAFC02E0641C75
:10245000600B0ED102213046FEF792FC0028F6D028
:102460000398C1B23046FEF7C8FC08E0641C600B5C
:1024700005D02868401C2860002005B0F0BD01216F
:102480003046FEF77DFC0028F0D00120F5E7000083
:102490008C0100200054004070B515460024022233
:1024A000FFF7B8FFE9B20C4D2846FEF7A6FC07E09F
:1024B000641C600B04D009490868401C086070BDAA
:1024C00040212846FEF75CFC0028F1D00121284677
:1024D000FEF74CFC70BD0000005400408C01002051
:1024E00010B5FFF70DFF10BD10B5FFF751FF10BD80
:1024F00010B5FFF787FF10BD10B5FFF7CDFF10BD7A
:10250000F0B5444C444D87B021682868FDF791FE32
:10251000286061686868FDF78CFE00240A27FF4385
:102520006860A600A8593946FDF706FF641CA8514B
:10253000032CF6DB39480024006804AF00903848CB
:10254000A60080590099FDF77CFE641CB851032C4D
:10255000F5DB344E049834682146FDF772FEB1680D
:10256000FDF76BFE019001990498FDF76AFE214684
:10257000FDF70EFE074601990598FDF762FE7168AA
:10258000FDF706FE044621460598FDF75AFE01991F
:10259000FDF753FEB06021460698FDF752FE39461E
:1025A000FDF74BFE3060069A01461046FDF749FEE6
:1025B0002146FDF7EDFD70601748FEF7FDFF1A4953
:1025C0001A4A4118914222D27F22D20501460024A4
:1025D0001046FDF773FE0090A700E959FDF731FEA4
:1025E000641CE851032C01DA0098F5E70B483F2101
:1025F0000906006800F005F907460024A0002958E4
:1026000080193A4600F0D5F8641C032CF6DB07B0BD
:10261000F0BD00008C030020740300206C0000203B
:1026200080030020E4000020CCCCCCC03233730007
:10263000F8B500250D4F01F021FA0024A6000A216B
:10264000B859C943FDF778FE01460948094A3018D0
:1026500000F0AFF8641C032CF0DB7D20C000FFF716
:10266000AEFA6D1C642DE6DBF8BD0000740300209B
:10267000E40000209A99593F10B50120FEF7B6FFFB
:1026800010BD0EB500226B461A805A8001911A8146
:102690009A726946FEF75AFD0EBD000070B50646F7
:1026A000FFF740FD194C21692061451A3046FDF7BE
:1026B000C2FE1749FDF7C5FD0646012120468907E0
:1026C0000C3000F063F82846FDF7B5FE05463046AD
:1026D0006168FDF7AEFD2946FDF7B3FD0D49FDF735
:1026E000B0FDE168FDF754FD0B49E060884205DD6F
:1026F000FF2000F039F87F20C00503E0FF2000F044
:1027000021F800206060002070BD0000B8000020AB
:102710008988883D6F12833A48E1FA3E70B50D46CC
:102720000446FFF7FFFC2146FDF7FAFC6C43200945
:10273000814203D90F2000F017F870BD0F2000F080
:1027400001F870BD70B50446064DC00703D00421E2
:102750002846FEF7FCFAA00703D508212846FEF715
:10276000F6FA70BD0000004870B50446064DC0077B
:1027700003D004212846FEF7E8FAA00703D5082174
:102780002846FEF7E2FA70BD0000004870B5044626
:102790000120C0070D4645400E462068FDF7BAFEF1
:1027A00000D2266028462168FDF7B4FE00D22560DD
:1027B00070BD70B505460C467F2016461146C00513
:1027C000FDF737FD2146FDF73CFD044631462868FC
:1027D000FDF737FD2146FDF7DBFC286070BD10B525
:1027E000FDF76CFD7F24E4052146FDF726FDA042A0
:1027F00001DD204610BD0121C9078842FAD9002019
:1028000010BD10B5FDF71DFD7F24E4052146FDF741
:1028100014FDA04201DD204610BD0121C9078842F8
:10282000FAD9002010BD00000EB57D20C000FFF7D2
:10283000C6F9FFF77BFC01F09DF901F0C7FAC74824
:10284000FFF7BDF9FFF74CFE00F0E6FF0021084658
:1028500001F05CF80021012001F058F8002103206C
:1028600001F054F80021022001F050F801F0D2F8F4
:1028700001F0BFF800282DD0FEF79EFDB8490120D9
:102880008872087101F079F8B64D00240020FEF737
:1028900009FE2968FDF77CFC28607D20C000FFF759
:1028A0008EF9641C402CF1DB0521C9432868FDF733
:1028B00043FD2860FFF756FC01F05EF8FFF7B8FE15
:1028C000FFF7A4FAFFF7AAFAA7480068002803D088
:1028D000072021E004201FE0FFF724FC6863FFF7D6
:1028E00021FCA04C0546606B281AFDF7A4FD20636F
:1028F000002802DC7F20C00520639C49FDF7A1FC75
:102900009B492063884201DD062005E09648656307
:102910000068142802DD0820FFF7EEF901F0AEF898
:10292000FFF7EEFDFEF742FF0020FEF7BBFD8D4CEA
:10293000E168FDF786FC06460120FEF7B3FD01467F
:102940008C4F20463A460C30FFF733FF8A486660CA
:1029500001683A466846FFF72CFF2046874A203038
:102960002168FFF726FF3A4631462046FFF721FF50
:102970000121C943206AFDF7DFFC06468049206833
:10298000FDF75FFC3146FDF754FC01907D48009C4B
:10299000844258DD734F786A0646FDF741FD794958
:1029A000FDF74FFC2146FDF74CFC0199FDF7F0FBCC
:1029B0006B49B4006C3108510646F86A002808D00B
:1029C000002030398200401C8E500C28FADB002099
:1029D000F86263486C490C300059FDF732FC0290F4
:1029E0005F483C3001593046FDF723FC0299FDF762
:1029F000CFFB5B493C310E51303908510146FDF7A0
:102A000020FC574E01469C36A019604AFFF7D1FEC4
:102A1000786A401C78620C2801DB002078623068FC
:102A20000290786A0B280ED10024A700F059029971
:102A3000FDF766FD04D2F05902904A48611C81629C
:102A4000641C0C2CF1DB474C2069002800D04D4859
:102A50004F49FDF79DFB0746A06AFDF7E1FC494E93
:102A60003146FDF7EEFB0099FDF7EBFB0199FDF711
:102A70008FFB3946FDF744FD03D346492068884261
:102A800001DA012000E000202061A06AFDF7C8FC07
:102A90003146FDF7D6FB0099FDF7D3FB0199FDF711
:102AA00077FBA0602069002801D0082108E03A489F
:102AB0000068002806D039480068002804D00F219B
:102AC00037482DE00C2113E06069002812D0E0693E
:102AD000002802D1FFF726FBE061FFF723FBE16945
:102AE000411A2F48814202D900206061E06108212B
:102AF0001A4815E0A069002815D0E069002802D125
:102B0000FFF710FBE061FFF70DFBE169411A244874
:102B1000814204D9A169491EA1610021E16103211B
:102B2000FFF7FCFD0AE00E48807A002803D0FF2062
:102B3000FFF71AFE02E0FF20FFF704FEFEF79CFD00
:102B40007D24E40002E00A20FFF739F8FFF7EAFAF3
:102B5000401BA04200D3C2E6F5E70000A0860100BA
:102B6000440200203C0000208C010020BD37863547
:102B70000AD7A33C492E7F3F3800002029EA7F3F37
:102B80000000A03FCDCCCC3D42F27C3F67B17F3FFF
:102B900000006040CDCC2C40940000209C00002020
:102BA00020A1070010B506490868002807D00020BA
:102BB0000860091D08710920C006FEF77EF810BDE7
:102BC0009001002070B504467F20C005844201DDDD
:102BD000044604E00120C007844200D900240949CA
:102BE0002046FDF72EFB054621460846FDF729FB4A
:102BF0000549FDF726FB2946FDF7CAFA0349FDF70B
:102C0000C7FA70BD7593583F7593183E0AD7A33B1A
:102C100005490868022804D001DA02200860401C37
:102C200070470020FAE70000440100200C49486882
:102C3000002804D0012807D002280AD10BE0084858
:102C40001C308860012003E005482830886002209D
:102C50004860401C70470248103088600020F7E749
:102C60004401002010B508494868401C486003280A
:102C700001DD00204860044849681430415C25208B
:102C800001F014F910BD00009400002010B5416857
:102C900000788007800DFF38FF3802380818FDF7EC
:102CA000BFFB0821C943FDF747FB10BDF1B54A48FA
:102CB00084B001680498494F494E8400002904D02B
:102CC00038594849FDF7BDFA3851474800250159A0
:102CD00042480C300059FDF713FC03D1305900284D
:102CE00000DD0125404801210059C90748403B4902
:102CF0000C310959FDF704FC04D131590120C007FA
:102D0000814226D8002D24D134480221183005599B
:102D10002846FDF711FB31493C310959FDF738FAD6
:102D200031590091FDF734FA3049FDF78AFA3049FC
:102D30000959FDF786FA2F490968FDF782FA3959D2
:102D4000FDF726FA385125483C30055124380099C2
:102D5000015125480C300159E019FFF717FD2448AF
:102D60000C3801593059FDF76CFA1C4E39590C36A4
:102D7000FDF70EFA039004983746C5001837E81996
:102D8000019000214068C943FDF7D6FA02901A4825
:102D900000210059C9430090FDF7CEFA0299FDF7D2
:102DA00048FA13490C310959FDF74BFA10491C39FF
:102DB000C968FDF746FA0399FDF73FFA30510198CB
:102DC000795941600098785107480159A019FFF7D7
:102DD000DDFC305905B0F0BD2C000020E4030020DC
:102DE000E801002048E17A3F243F00087EAA2A3EFD
:102DF000600100206C0000208003002010B5044812
:102E000001680448FDF75AFA0349C86010BD000084
:102E10006C00002017B7513B44010020F0B51FB4EF
:102E200096B084460C460246199D189803904900B6
:102E300068006300490840080193002A01D0012678
:102E400000E000269E19FE4BF6185B109E422BD325
:102E50006E00039F0296002F00D00127F719F84E4D
:102E6000F84BBE199E421FD3039E0346F64F3343D1
:102E700009D03B469C4201D1002A04D0019B002A84
:102E800005D0012604E0002039461BB0F0BD002625
:102E90009E19EE4B9E4207D8039F029E002F00D042
:102EA0000127F6199E4207D92B4660462146189AFB
:102EB000FEF714FA1BB0F0BD0023002C29DAE44E13
:102EC000B04226DAE34EB04201DB022321E0DE4EBF
:102ED000B0421EDBE04E070DBE19142E09DD34276B
:102EE000BF1B039EFE400196BE40039FBE420BD017
:102EF0000FE0039F002F0CD11427BF1B0646FE4096
:102F00000196BE40864204D1019BDE07F60F0223E4
:102F10009B1B0E46164318D1002D16DA002C03D049
:102F2000022B01D0012B06D00220FEF707FAFEF794
:102F3000CBF91BB0F0BD0220FEF700FAFEF7C4F992
:102F40000122D20751401BB0F0BD039E002E61D17B
:102F5000BF4EB04220D1C148844201D1002A08D0DE
:102F6000B948814209DB002D10DB189829461BB0B7
:102F7000F0BD0020B4491BB0F0BD002D06DA0122DF
:102F80002946D207189851401BB0F0BDB449794486
:102F9000086849681BB0F0BDAB4FB84225D1002D81
:102FA0001FDA002904D0B14212D1002A09D018E05A
:102FB000002A72D1A649E20F0020D20711431BB0AC
:102FC000F0BD0020E20F0146D20711431BB0F0BD57
:102FD000B14206DA234600203946FDF7F7FB1BB065
:102FE000F0BD104621461BB0F0BDB14212DA0126F9
:102FF000B607B54203D1234610461946FEE3994E63
:10300000B54207D1261E05DB1046314600F01CFEF6
:103010001BB0F0BD67007F081646002A40D100298A
:103020000AD08B4A914229D1002C0EDD002D1CDBE9
:10303000002011461BB0F0BD022B16D0002C14D07E
:10304000012B12D1002C14DB0FE0002C28DA002D0C
:1030500009DB012B03D000207D491BB0F0BD00200F
:1030600081491BB0F0BD012B03D0002001461BB0ED
:10307000F0BD00200121C9071BB0F0BD724A91428A
:103080000ED1002C01DA002B17D0022B06D0002025
:10309000C043FDF729FC1BB0F0BD90E20120F8E72A
:1030A000E217521C94461A4307D000220892664C3D
:1030B00062465B1E1A4307D009E00120FEF73EF985
:1030C000FEF710F91BB0F0BD0022644C0892674A6D
:1030D00090427DDD664B674A98421FDD914202DCDB
:1030E000002D05DB4DE05848814217DB002D48DDFF
:1030F0000220FEF723F9FEF7FDF805460E460022F2
:10310000534B21460898FDF723F9084671004908FA
:10311000C00FC007014328461BB0F0BD914215DA2D
:10312000002D2EDA0220FEF709F9FEF7E3F8054636
:103130000E460022464B21460898FDF709F9720019
:103140005208C80FC0070243114617E03E4B994290
:1031500023DD002D15DD0220FEF7F0F8FEF7CAF89A
:1031600005460E4600223A4B21460898FDF7F0F836
:10317000084671004908C00FC007014328461BB02C
:10318000F0BD0220FEF7DAF8FEF7BEF84900490864
:10319000E20FD20711431BB0F0BD00223046394682
:1031A000FDF706FB012205460E46D243FDF786FBDE
:1031B000314A324BFDF702FB2A463346FDF7C8F889
:1031C0000022284BFDF7FAFA07462A46334600E06C
:1031D00064E0039110461946FDF7BAF83A46039B9E
:1031E000FDF7B6F80746032209915207244B2846FB
:1031F0003146FDF7ADF807910C90224A204B384636
:103200000999FDF7A5F8074601911F4A1F4B28466B
:103210003146FDF79DF83A46019BFDF7C9FA07468E
:103220000B460246099107990C98FDF71DFA0025F7
:103230000E462846079B0C9AFDF7BAFA3A4627E055
:10324000FFFF1F00FFFF0F000000F03F0000E0FF46
:103250000000F07F0000404301FCFFFF0000F0BFD2
:10326000361000000000E03F0000F0FF0000E041E9
:103270000000F043FFFFEF3F555555555555D53FDD
:103280004715F73FFE822B6544DF5DF80BAE543ED9
:10329000099BFDF793FA02460B4652E101250020F7
:1032A0002D05A94207DA352230463946FDF706FBDF
:1032B00006463420C0430A151218FE481018039021
:1032C0000803FD49000B01430F46FC49884201DC1D
:1032D000002003E0FA49884202DA0120119005E05B
:1032E000002011900398401C7F1B039011980597B4
:1032F000C200F4480F927844801843680268394647
:1033000030460D930292FDF753FA07910C90304628
:103310000D9B029A0599FDF7A7F902460B4600207E
:10332000E549FDF753FA09910490079B0C9AFDF7C4
:103330000FF8129000201090E3480D467844006882
:103340000E90012178104907084311990D9B8904BB
:1033500040180121C90447183946029A0E98FDF712
:1033600027FA3246059BFDF729FA02460B46294605
:103370001098FCF7EDFF064602913B4629460E9A4F
:103380001098FCF7E5FF079B0C9AFDF717FA3246F9
:10339000029BFDF70DFA099B049AFCF7D9FF0591F2
:1033A000129A0A902B4610461946FCF7D1FF0646A2
:1033B0000246C6480F460B4606217844FDF72EFF0D
:1033C00032463B460091049010461946FCF7C0FF78
:1033D000009B049AFCF7BCFF06460F462B46194695
:1033E000129A1098FDF740F9059B0A9AFCF7B0FF76
:1033F00032463B46FDF738F9109A079104902B4668
:1034000010461946FCF7A4FFB14E0022334609913D
:103410000290FDF729F9079B049AFDF725F9002092
:103420000746024633460091FDF7C2F9099B029A0E
:10343000FDF7BEF9079B049AFDF7C0F906460D910A
:103440003A462946009B1098FCF782FF07910C90A2
:103450002B463046129A0D99FCF77AFF05460E4628
:103460003A46009B05990A98FCF772FF33462A46B4
:10347000FDF7FAF802460B460746099107990C98A2
:10348000FDF7F2F800250E462846079B0C9AFDF73B
:103490008FF93A46099BFDF791F9074607220991F2
:1034A00052078C4B31462846FCF752FF079100909B
:1034B000894A884B38460999FCF74AFF074601912B
:1034C000864A874B31462846FCF742FF3A46019B25
:1034D000FDF7CAF8834B7B440F9A9B181A685B6808
:1034E000FDF7C2F8029009910398FDF7FDF90591E7
:1034F0000490099B029A07990098FDF7B5F87A4B5A
:103500007B440F9A9B181A685B6817460393FDF774
:10351000ABF8059B049AFDF7A7F80E462846059BD5
:10352000049AFDF745F93A46039BFDF741F9079BDD
:10353000009AFDF73DF9099B029AFDF73FF9024613
:103540000B46199900200C900F461898FCF700FFC5
:10355000029104903B460C9A19991898FDF728F9A6
:103560002A463346FCF7F4FE029B049AFDF77CF8EA
:1035700009910E902A46334639460C98FCF7E8FE2E
:1035800006460F46099B0E9AFDF76EF8574A0D4600
:10359000914220DB5242AA18024310D132463B46E8
:1035A000FDF706F904900391514A524B09990E9880
:1035B000FDF75AF8039B049AFCF772FF1ED2022013
:1035C000FDF7BCFEFDF796FE49004908E20FD20761
:1035D00011431BB0F0BD6A00474B52089A420DD30D
:1035E000464AAA18024300D0CBE532463B46FDF7D7
:1035F000DFF8099B0E9AFCF753FFF5D9680000230A
:1036000040082C490393020D3D4B5218984223DD8C
:1036100001200005521CD04042195000400D4018B6
:1036200038497944096813468C463749C1408B4371
:1036300012030121120B090551181422101AC1405E
:103640000391002D01DA4842039062463046394624
:10365000FDF7AEF806460F4632463B4609990E98EE
:10366000FDF702F800252A46284B28460591FCF76D
:103670006FFE07910C90264A264B28460599FCF7C9
:1036800067FE0091029032463B4628460599FDF7B9
:103690008FF8099B0E9AFDF791F81F4A1F4BFCF714
:1036A00057FE009B029AFCF7DFFF07460B460246D7
:1036B000099135E001FCFFFF0000F03F8E98030008
:1036C0007AB60B00460C0000880C0000B20B00001C
:1036D0000000084009C7EE3FFD033ADCF5015B142A
:1036E000E02F3EBE860A00004C0A00000000904019
:1036F000FE822B654715973C00CC904000346F3F0D
:103700000000E03FA2090000FFFF0F00432EE63F4C
:10371000396CA80C615C20BEEF39FAFE422EE63F00
:1037200007990C98FCF7A0FF05460E46079B0C9ADC
:10373000FDF73EF83A46099BFDF740F809912A4605
:1037400033460E9010461946FCF702FE0746024625
:103750002F480B46059105217844FDF75FFD3A4659
:10376000059BFCF7F5FD2A463346FDF727F807468B
:10377000019128463146099B0E9AFCF7E9FD099B09
:103780000E9AFCF771FF012304910C9000229B0715
:1037900038460199FDF70CF805910E903A462846F7
:1037A0003146019BFCF7D4FD059B0E9AFDF70EF800
:1037B000049B0C9AFCF7FCFF2A463346FCF7F8FF03
:1037C0000022144BFCF7FAFF064603980D4600054D
:1037D00041190915002912DC30462946039AFDF7E4
:1037E0006DF8FDF705FD042801D1FDF78DFD30468C
:1037F0002946039AFDF762F8064601E004E029181D
:103800000B46324621460898FCF7A2FD1BB0F0BDDE
:10381000440800000000F03FFEB5022569460D7126
:103820000320487100248C71CC7101212846FDF7DA
:103830002DFB314F31483946FEF723FF01210E029F
:103840003046FDF723FB39462D4F3846FEF719FF6A
:103850002C4860210180012141808481068284609E
:1038600010200924E406009069462046FDF725FA59
:10387000042211462046FDF758FA22493846FDF742
:10388000ADFB4020009069462046FDF716FA012264
:1038900006212046FDF749FA1A491848FDF79EFB14
:1038A0008020009069462046FDF707FA0122072193
:1038B0002046FDF73AFA13491048FDF7CDFB124CAC
:1038C000694620460095FDF7F8F901221146204689
:1038D000FDF72BFA0B490948FDF706FC01210748C3
:1038E000FDF766FB01210548FDF76CFB0121384619
:1038F000FDF75EFBFEBD0000CF07000000040040A6
:10390000002000402C0400200004004810B50A46A6
:10391000044612491046FCF794FCFCF793FD00287E
:1039200001DA002003E00E49884200DD0846002C41
:1039300009D0012C0CD00B49022C0CD0032C01D146
:1039400080B2886310BD074980B24031086010BD65
:1039500080B2054900E080B2486310BD00E0F94440
:10396000CF070000000400400020004010B5FEF723
:103970007DF9FEF72FF910BD704700B585B0142111
:103980006846FCF7EAFB684600F0A1FA0021012036
:1039900000F08CFA0121022000F088FA01210620B3
:1039A00000F084FA0F21112000F080FA0021042099
:1039B00000F07CFA0321084600F078FA20211D204F
:1039C00000F074FA00F0D0F8FD2000F011F90020AA
:1039D00000F00EF900F0C2F8E22000F035FA002104
:1039E000052000F063FA8F21002000F05FFA05B097
:1039F00000BD10B575216820FEF77AFD682807D054
:103A0000982805D07D2803D0722801D0002010BD51
:103A1000012010BD10B580226B216820FEF76CFDDF
:103A20001548FEF7CCF801226B216820FEF764FDF3
:103A300075216820FEF75CFD682801D0012400E0B4
:103A400000246420FEF7BBF818221C216820FEF732
:103A500053FD002C04D005221D216820FEF74CFDEB
:103A600018221B216820FEF747FD03221A21682037
:103A7000FEF742FD10BD0000409C0000F0B593B081
:103A80000E236A463B216820FEF72EFD029803991B
:103A90000002401800B2FCF7C3FC2D4C20600098D7
:103AA00001990002401800B24042FCF7B9FC606086
:103AB000049805990002401800B2FCF7B1FCA06020
:103AC000089809990002401800B2FCF7A9FC11906F
:103AD0000A980B990002401800B2FCF7A1FC109064
:103AE0000C980D990002401800B2FCF799FC129056
:103AF000243421681098FCF79CFB109061681198A1
:103B0000FCF797FB1190A1681298FCF792FB1290BA
:103B10000120109AC007119942401091114641406E
:103B2000119112990A4F4140002410AE0C371291A6
:103B3000A50070590749FCF784FB0749FCF781FB96
:103B40007051641C7851032CF2DB13B0F0BD0000FF
:103B50007403002000007A3D35FA8E3C01490120B3
:103B600088617047001400480149012008817047AE
:103B700020140048FEB501246846047100258571B3
:103B8000C4710326467102200B4F009069463846E7
:103B9000FDF793F8694638460094FDF78EF807481C
:103BA000046005718571C471467101460920C00623
:103BB000FDF783F8BC61FEBD0014004894010020AD
:103BC00070B4002007210223074C0925074EED069B
:103BD000A3614200288A3381C007C00F1043491EE9
:103BE000F6D570BC7047000000140048201400484F
:103BF000F8B504460F4809260168F6060125002994
:103C000006D105600C48057101463046FDF755F8B0
:103C100007210A4B0A4F022022460A41D20701D04F
:103C2000B56100E01D81B861064A1081491EF3D5D7
:103C3000F8BD000090010020940100202000004801
:103C40000014004820140048F8B506460C46FCF75E
:103C5000A5FE051E0F4600D00120014349000B4878
:103C60004908411AC90F0DD0002E01D0012100E0F2
:103C700000210C4361004908401AC00F02D1012005
:103C8000FDF75CFB28463946F8BD00000000F07FD8
:103C9000F8B5464E464D31682868FCF731FC04D132
:103CA00071686868FCF72CFC54D034682C6070682C
:103CB000404E68603146FCF7C4FA3F4F3946FCF786
:103CC000C0FA054631462046FCF7BBFA3946FCF7F8
:103CD000B8FA0646FEF73CF8354C08342060284612
:103CE000FEF736F860602846FEF728F805463046AD
:103CF000FEF724F82946FCF7A4FA0646A06060689F
:103D00000146FCF79EFA054620680146FCF799FA41
:103D10002946FCF73DFA2949054688420FDD314620
:103D20000846FCF78EFA7F21C905FCF786FA0146A2
:103D30002846FCF7C3FAFDF773F8054600E0204D6E
:103D400020682946FCF77DFA206029466068FCF768
:103D500078FA6060164C1B4E0834A06800907068BA
:103D60000099FCF76EFAB768054661683846FCF7BB
:103D700068FA2946FCF75DFA134D686030680099CF
:103D8000FCF75FFA064638462168FCF75AFA3146D6
:103D9000FCF74FFA7F24E405286021462846FEF709
:103DA000F5FC2146281DFEF7F1FCF8BDF4010020CA
:103DB000D000002000008C4235FA8E3C6F12833A0E
:103DC000F4FD343FE4000020A403002010B50848AF
:103DD000064941610749CA6903231202120A4404D1
:103DE0002243CA6100218161036110BD7F8D5B00A8
:103DF00000E000E004ED00E010B509484269816987
:103E0000084C2068814201D2401A01E0521A101871
:103E100021600621FCF784F961684018606010BDDC
:103E200000E000E09C010020064A10B580008018E8
:103E3000FCF7FCFE042804D0FCF7F0FE0520FDF79B
:103E40005BFF10BD007C000810B50446FFF78CFE38
:103E50002046FFF7CDFEFFF781FE002010BD70B5B4
:103E60000D4606460024FFF77FFE6120FFF7C0FEE7
:103E7000FEF798FE04E0FFF7A3FEA1007050641C5B
:103E8000AC42F8DBFFF76AFE70BD10B5C406E40E65
:103E9000FFF76AFE2046FFF7ABFEFEF783FEFFF753
:103EA0008FFE0446FFF75AFE204610BD70B584060B
:103EB000A40E20200D460443FFF756FE2046FFF7D0
:103EC00097FE2846FFF794FEFFF748FE70BD70B5D9
:103ED00005460024FFF748FE2A20FFF789FEA000D0
:103EE0002858FFF785FE641C052CF8DBFFF736FE2B
:103EF00070BD0C0100010003000C02000200030071
:103F00000C0300030003000C0400030004000C0475
:103F100000030003000C0400030002000C04000373
:103F200000010000CDCC4C3FCDCC4C3F0000003F09
:103F3000CDCC4C3FCDCC4C3F0000003F00000000FA
:103F4000000000000000F03F000000000000F83F0B
:103F500000000000000000000000004003B8E23F45
:103F6000000000000000000006D0CF43EBFD4C3EF7
:103F7000033333333333E33FFFAB6FDBB66DDB3FEC
:103F80004D268F515555D53F01411DA96074D13F34
:103F900065DBC9934A86CD3FEF4E454A287ECA3F2E
:103FA0003E5555555555C53F93BDBE166CC166BFB0
:103FB0002CDE25AF6A56113FF16BD2C541BDBBBEA9
:103FC000D0A4BE726937663E000000000000000009
:103FD000F43F000800000020E80100003E0A00084D
:103FE00058400008E8010020580600002C13000883
:103FF00059D3FFFFC132010518CDCC4C3E292029F1
:1040000004C12D6666864004210B12803F1CA93C2A
:10401000A1035820C1A0097B14524185EB41410BFB
:1040200014803F0C01245AE0C07A60C8011C13546C
:104030000142202DB81E053E0438089A99193FAE5A
:1040400047610428099A99993ECDCC0C3F04692C0C
:084050001A60045A6C3401608F
:04000005080000C926
:00000001FF
